:100000000C9450010C946D010C946D010C946D01D5
:100010000C946D010C946D010C946D010C946D01A8
:100020000C946D010C946D010C946D010C9475028F
:100030000C946D010C946D010C946D010C946D0188
:100040000C942B020C946D010C946D010C946D01B9
:100050000C946D010C946D010C946D010C946D0168
:100060000C946D010C946D01000000002500280027
:100070002B0000000000240027002A0004040404D0
:100080000404040402020202020203030303030342
:10009000010204081020408001020408102001021F
:1000A00004081020898A56D55DED0C3A69353795DC
:1000B000DDA864D4CD4C4EEB8311771747A557DAF2
:1000C000DC4CA5148DDBB030735C2056B2D2DC71F1
:1000D000C9798C6C5126096229AACD68372846F166
:1000E0002173DAF89C4547384E8362356DE1C405CB
:1000F0004AD5A4836D372ED6324F9552B8D82BDC13
:10010000D84A607D0B76E3FA8E565DB5C3D2058A78
:1001100097F4AA8C1B08513CA73C712382CDE8249C
:10012000A783C822729CEC36B24AF1134ED3A8A220
:100130003B8A386981529E1D0E29418D7D77C56CA1
:10014000872FF6CD620FDDC654668ACD4E13B3AB52
:100150001E14374D4CAA72886A1731EA8E219C937F
:100160004463C653B88E8370BA74E7340EC275C345
:100170008CBA2448848A524ED28410DA93386E1393
:1001800062D84C253B8D8F71B284ED143EA6A91226
:10019000565CF898BB53C54EE393ED4C96A8857317
:1001A0006AC28D9314D6EB6D378A1D2061A7C3A94F
:1001B000898150BF36B7D60242FB42D2972808B792
:1001C0004B4F4F9C9840AA7B3C55A058FAB498D40A
:1001D00089D2F22B35D2343AB1A962913B98A4AAC4
:1001E00082C26E6392DF0C163B854D69A6D52D2722
:1001F00021E5D9D61013EC3876D2CCAEB353DA0A57
:10020000C348C94AA9345C4C952ABEF04D93DA9490
:1002100038DAB25C4A52426DAAE43849092DB18BF2
:10022000E22625E6A46E8C5794984D3B284A5152FD
:10023000165BA7A8458D49CA5DE4943F3A496F977C
:10024000529460CD2BC54A53A2B39CC4A8458B3AA7
:100250002317AD24C6BBC80CB49D186F33B3C97641
:10026000B1BD710F67D9C53156DD55152FBB2BE6D2
:1002700074B535EC6EC432584E71A2F43455DBC5FA
:1002800075C65D556515D7D8705393551CEFD24D83
:100290005576B1AD093735D9CE52CAD5DC153F00F8
:1002A00011241FBECFEFD8E0DEBFCDBF12E0A0E02B
:1002B000B1E0EAEEFCE002C005900D92A436B10771
:1002C000D9F722E0A4E6B2E001C01D92A639B20738
:1002D000E1F70E94F6040C9473060C940000CF938F
:1002E000DF93A0919202B0919302FD014491429557
:1002F000942F9373F4E09F9F900111244C7C4695BA
:100300004695242B922F9575990F2A7A2695292B9D
:1003100030E0322F222770919402C82FD0E0AE0136
:10032000470F511D49305105B4F0FD0131964491FC
:10033000642F6295962F9373E4E09E9FA001112491
:100340006C7C66956695462B942F9575990F4A7A25
:100350004695492B242B072E02C0220F331F0A94E7
:10036000E2F740E150E04C1B5D0B02C0369527954B
:100370004A95E2F7780F783018F47093940208C029
:100380007850709394021196B0939302A0939202C6
:10039000822FDF91CF9108953FB7F89480917F022B
:1003A00090918002A0918102B091820226B5A89B13
:1003B00005C02F3F19F00196A11DB11D3FBFBA2FF7
:1003C000A92F982F8827820F911DA11DB11DBC0157
:1003D000CD0142E0660F771F881F991F4A95D1F71C
:1003E00008958F929F92AF92BF92CF92DF92EF9239
:1003F000FF926B017C010E94CC014B015C01C11496
:10040000D104E104F104F1F00E94CC01DC01CB0144
:1004100088199909AA09BB09883E9340A105B1052D
:1004200070F321E0C21AD108E108F10888EE880EC5
:1004300083E0981EA11CB11CC114D104E104F10495
:1004400019F7DDCFFF90EF90DF90CF90BF90AF9086
:100450009F908F9008951F920F920FB60F921124C4
:100460002F933F938F939F93AF93BF9380917B0282
:1004700090917C02A0917D02B0917E0230917A022F
:1004800023E0230F2D3720F40196A11DB11D05C0D7
:1004900026E8230F0296A11DB11D20937A028093B6
:1004A0007B0290937C02A0937D02B0937E028091A8
:1004B0007F0290918002A0918102B0918202019608
:1004C000A11DB11D80937F0290938002A0938102B1
:1004D000B0938202BF91AF919F918F913F912F91E5
:1004E0000F900FBE0F901F9018951F920F920FB68E
:1004F0000F9211242F923F924F925F926F927F92B0
:100500008F929F92AF92BF92CF92DF92EF92FF9223
:100510000F931F932F933F934F935F936F937F930B
:100520008F939F93AF93BF93EF93FF93CF93DF93FB
:10053000CDB7DEB7A497DEBFCDBF8091790280939F
:10054000B400789490918302992309F18091780204
:10055000891720F48F5F8093780202C0109278028E
:10056000E0917802E93288F5F0E0EE5FFE4FA0817D
:1005700020919002309191020A2E000CBB0B0E9438
:100580006C06BB27A92F982F872FBC0120C0209174
:10059000000130910101C90196958795A90141702B
:1005A000552720FF02C040E058EB84279527909301
:1005B000010180930001609190027091910280FD91
:1005C00006C071956195710902C060E070E0E0912C
:1005D00085024E2FEE0F550B5AA349A3609074026B
:1005E00070907502409184022091760230917702DA
:1005F0004203C001439F900D1124880F892F881F4B
:10060000990B681B790BE9A1FAA1E69DC001E79D52
:10061000900DF69D900D1124880F892F881F990B3E
:100620004B01881A990A40908602042C000C550848
:1006300040917202509173025A834983449EC001D3
:10064000459E900D549E900D1124880F892F881F70
:10065000990B1401281A390A80918702E82F880F14
:10066000FF0BFC83EB8340917002509171025E831B
:100670004D83E49FC001E59F900DF49F900D1124E0
:10068000880F892F881F990BF101E81BF90BF88758
:10069000EF8380918802482F880F550B5A8749872E
:1006A000E0916E02F0916F02FC87EB874E9FC001D4
:1006B0004F9F900D5E9F900D1124880F892F881FEA
:1006C000990B4F815885481B590B5E874D87809148
:1006D0008902E82F880FFF0BF88BEF8740916C029F
:1006E00050916D025A8B498BE49FC001E59F900D9C
:1006F000F49F900D1124880F892F881F990BED8589
:10070000FE85E81BF90BFC8BEB8B80918A02482F4E
:10071000880F550B5E8B4D8BE0916A02F0916B0256
:10072000F88FEF8B4E9FC0014F9F900D5E9F900DF5
:100730001124880F892F881F990B4B895C89481BCE
:10074000590B5A8F498F80918B02E82F880FFF0B2E
:10075000FC8FEB8F40916802509169025E8F4D8F44
:10076000E49FC001E59F900DF49F900D1124880F28
:10077000892F881F990BE98DFA8DE81BF90BF8A3D7
:10078000EF8FA0908C02B0908D02E0906602F09006
:1007900067029501D7010E945506DC01CB014FE0AD
:1007A000B595A795979587954A95D1F76F01C81A82
:1007B000D90A00918E0210918F02409164025091EB
:1007C00065025CA34BA39801DA010E945506DC0187
:1007D000CB015FE0B595A795979587955A95D1F789
:1007E000A601481B590B411562E056073CF4411520
:1007F0007EEF57072CF440E05EEF02C04FEF51E070
:10080000E9A1FAA1E89DC001E99D900DF89D900D28
:100810001124880F892F881F990B860D971D90939F
:10082000770280937602429CC001439C900D529CBB
:10083000900D1124880F892F881F990BE981FA8167
:100840008E0F9F1F9093750280937402EB81FC8141
:100850002F813885E29FC001E39F900DF29F900D9C
:100860001124880F892F881F990BED81FE818E0F2F
:100870009F1F9093730280937202E985FA852D85FC
:100880003E85E29FC001E39F900DF29F900D1124E1
:10089000880F892F881F990BEB85FC858E0F9F1F72
:1008A0009093710280937002EF85F8892B893C89BF
:1008B000E29FC001E39F900DF29F900D1124880FDD
:1008C000892F881F990BE989FA898E0F9F1F9093B2
:1008D0006F0280936E02ED89FE89298D3A8DE29F29
:1008E000C001E39F900DF29F900D1124880F892F76
:1008F000881F990BEF89F88D8E0F9F1F90936D02C3
:1009000080936C02EB8DFC8D2F8D38A1E29FC0018E
:10091000E39F900DF29F900D1124880F892F881F5F
:10092000990BED8DFE8D8E0F9F1F90936B02809320
:100930006A029501D6010E945506DC01CB012FE029
:10094000B595A795979587952A95D1F7B701680F23
:10095000791F70936902609368029801DA010E941E
:100960005506DC01CB013FE0B595A7959795879596
:100970003A95D1F7EBA1FCA18E0F9F1F90936702D0
:1009800080936602509365024093640255954795A3
:1009900055954795405840937902A4960FB6F89420
:1009A000DEBF0FBECDBFDF91CF91FF91EF91BF9121
:1009B000AF919F918F917F916F915F914F913F91F7
:1009C0002F911F910F91FF90EF90DF90CF90BF90EC
:1009D000AF909F908F907F906F905F904F903F90DF
:1009E0002F900F900FBE0F901F901895789484B59C
:1009F000826084BD84B5816084BD85B5826085BD1B
:100A000085B5816085BD80916E00816080936E00A8
:100A1000109281008091810082608093810080919A
:100A2000810081608093810080918000816080934B
:100A300080008091B10084608093B1008091B0000B
:100A400081608093B00080917A00846080937A0006
:100A500080917A00826080937A0080917A00816030
:100A600080937A0080917A00806880937A00109257
:100A7000C10003E910E06FE7E62E60E0F62ED3E256
:100A8000C1E070EDC72E77E0D72EE0E0AE2EE0E0BB
:100A9000BE2EF4EA8F2EF0E09F2E49E0742E52E035
:100AA000652E60ED77E080E090E00E94F10180919A
:100AB000950281112FC0F8012491F70184918823B8
:100AC00099F090E0880F991FFC01EE58FF4FA59117
:100AD000B491FC01E859FF4F859194918FB7F89438
:100AE0009C91292B2C938FBFD093B000C093B10061
:100AF0001092700010928000709281001092850018
:100B000010928400D0928900C092880060926F0099
:100B1000C093950290929302809292021092940256
:100B200084E00E946F01582E811105C0109291023D
:100B300010929002AAC0FFE08F131DC01092910284
:100B40001092900210928F0210928E0210928D02DB
:100B500010928C0210928B0210928A0210928902DB
:100B600010928802109287021092860210928502DB
:100B7000109284028AC0E82FF0E0ED5AFD4F808188
:100B800090E0909391028093900281E00E946F0127
:100B9000382E86E00E946F01E82FF0E0ED5EFD4FF9
:100BA000408040928302311070C085E00E946F0146
:100BB000E82FF0E0EE0FFF1FED52FE4F8081918194
:100BC00090938F0280938E0285E00E946F01E82F40
:100BD000F0E0EE0FFF1FED56FE4F80819181909364
:100BE0008D0280938C0284E00E946F01E82FF0E078
:100BF000ED57FE4F808180938B0284E00E946F014D
:100C0000E82FF0E0ED58FE4F808180938A02442067
:100C1000E1F184E00E946F01E82FF0E0ED59FE4F12
:100C200080818093890284E00E946F01E82FF0E0C8
:100C3000ED5AFE4F80818093880284E00E946F010C
:100C4000E82FF0E0ED5BFE4F80818093870283E028
:100C50000E946F01E82FF0E0E55CFE4F80818093F9
:100C6000860283E00E946F01E82FF0E0ED5CFE4F0A
:100C700080818093850283E00E946F01E82FF0E07D
:100C8000E55DFE4F80818093840269E170E080E041
:100C900090E00E94F1018FE0581242CFA114B104FC
:100CA00009F4FFCE0E940000F8CE0E945D063323B7
:100CB00012F48A1B9B0B0C946E06A29FB001B39F8B
:100CC000C001A39F700D811D1124911DB29F700D55
:100CD000811D1124911D08950E945D06B7FF08959E
:0A0CE000821B930B0895F894FFCFD8
:100CEA000100002AD432B212251402E1C5025F5A69
:100CFA00050F26FCA5A5D6DDDCFC252B22210FFF3E
:100D0A00F8EEEDEFF7F6FA00030201CDDFF1041673
:100D1A00203B4DC0D4E8FC1025394DC0D8F0071F40
:100D2A00374F66B3BFCBD7E3EFFB07131F2B37430E
:100D3A004F5A66C0CBD6E1ECF7030E19242F3A4579
:100D4A00505B66AEBAC5D1DDE8F4FF0B17222E3927
:100D5A0045515CAEBCCAD8E6F4010F1D2B39475584
:100D6A0063717E929FADBAC8D5E3F0FE0B192634A3
:100D7A00414F5C00AE80B480BB40C380CB40D4C03E
:100D8A00DD80E780F1C0FB00064010401A002440D5
:100D9A002D0036403EC045C04C00538058C05D40CF
:100DAA00624066C069C06C806FC071C07380750094
:100DBA0077807EC0828083C0834084C0844085005F
:100DCA0086808780888089C08A008C408D008FC089
:100DDA0090C092009940A180AB40B840C7C0D8C02B
:100DEA00EB000040144027C038C0478054C05E0062
:100DFA0067406D00101112131415161718191A1BD3
:100E0A001C1D1E1F202122232425262728292A2BA0
:100E1A002D2F31333536393B3D3F424547494D4FFA
:100E2A005155575C5F63666A6E73777B80858A8FDC
:100E3A00959AA00002030405070A0F1420293951C4
:040E4A0072A1FF0092
:107E0000112484B714BE81FFF0D085E080938100F7
:107E100082E08093C00088E18093C10086E0809377
:107E2000C20080E18093C4008EE0C9D0259A86E02C
:107E300020E33CEF91E0309385002093840096BBD3
:107E4000B09BFECF1D9AA8958150A9F7CC24DD24C4
:107E500088248394B5E0AB2EA1E19A2EF3E0BF2EE7
:107E6000A2D0813461F49FD0082FAFD0023811F036
:107E7000013811F484E001C083E08DD089C08234E0
:107E800011F484E103C0853419F485E0A6D080C0E4
:107E9000853579F488D0E82EFF2485D0082F10E0AE
:107EA000102F00270E291F29000F111F8ED06801E7
:107EB0006FC0863521F484E090D080E0DECF843638
:107EC00009F040C070D06FD0082F6DD080E0C81688
:107ED00080E7D80618F4F601B7BEE895C0E0D1E017
:107EE00062D089930C17E1F7F0E0CF16F0E7DF06D8
:107EF00018F0F601B7BEE89568D007B600FCFDCFD4
:107F0000A601A0E0B1E02C9130E011968C91119780
:107F100090E0982F8827822B932B1296FA010C0160
:107F200087BEE89511244E5F5F4FF1E0A038BF0790
:107F300051F7F601A7BEE89507B600FCFDCF97BE46
:107F4000E89526C08437B1F42ED02DD0F82E2BD052
:107F50003CD0F601EF2C8F010F5F1F4F84911BD097
:107F6000EA94F801C1F70894C11CD11CFA94CF0C13
:107F7000D11C0EC0853739F428D08EE10CD085E9AC
:107F80000AD08FE07ACF813511F488E018D01DD067
:107F900080E101D065CF982F8091C00085FFFCCF94
:107FA0009093C60008958091C00087FFFCCF809118
:107FB000C00084FD01C0A8958091C6000895E0E648
:107FC000F0E098E1908380830895EDDF803219F02E
:107FD00088E0F5DFFFCF84E1DECF1F93182FE3DFCA
:107FE0001150E9F7F2DF1F91089580E0E8DFEE27F6
:047FF000FF270994CA
:027FFE00040479
:0400000300007E007B
:00000001FF
